:100000008528831203137F087F0403190C28FF033C
:100010007F0A0319FF030128080083120313220833
:10002000230403192E28A40104308312031324028D
:1000300003182728A501883083120313250203180B
:100040002328A50A1B2883120313A40A1428831249
:100050000313A203220A0319A3030D280800FA3090
:1000600083120313A200A3010D20FA30831203139D
:10007000A200A3010D20FA3083120313A200A301F2
:100080000D20FA3083120313A200A3010D2883125E
:100090000313A0001430A200A3010D20F03083123E
:1000A00003132005A100210E0F39A10021088700AC
:1000B00085110515851685120F302005A100210830
:1000C0008700851105158516851208008312031314
:1000D000A0000A30A200A3010D20F0308312031308
:1000E0002005A100210E0F39A100210887008511EC
:1000F0000511851685120F302005A1002108870003
:1001000085110511851685120800831603138116C3
:10011000011681158312810185010E3083169F001F
:10012000D130850083129F111F129F121F14831656
:100130009F173F3083128600EF30831686008312AC
:100140008701C030831687008312051185114C305A
:10015000A2000430A3000D20033083120313870094
:10016000851685120A30A200A3010D2003308312E8
:1001700003138700851685120A30A200A3010D2003
:100180000330831203138700851685120A30A200FC
:10019000A3010D20023083120313870085168512F8
:1001A0000C30662001306620013066204730472041
:1001B0006F304720203047204F3047206C30472099
:1001C000693047206D304720653047207830472020
:1001D000213047204C3047204330472044304720CF
:1001E0002D3047204F3047204B30472010308312AE
:1001F0000313A2002730A3000D2001306620630006
:0202000085284F
:02400E00323F3F
:00000001FF
